:020000040000FA
:100000003F0A490852084308760831082E0831088B
:100010004D08200862087908200841086C08650826
:10002000780841084C084208200861086C086208FA
:100030004008630872086F08770864082E08720881
:1000400075082008280843082908430852084F0863
:10005000570844082008520875087308730869088F
:1000600061082C082008500865086E087A086108A5
:0A007000200832083008300832087A
:04007A000008000872
:02007E0025005B
:10008000CF0C0200080C060070008604A604740A57
:100090000F024306740A010C8F0043065A0A020C31
:1000A0008F004306670A740A8604A6047000710074
:1000B0007200740A10024306620A010C90004307A2
:1000C000540A8605010C300071007200740A100297
:1000D00043066F0A020C90004307540AA605020C5F
:1000E000300071007200740A00000000000000007F
:1000F0000400F103F200B202D206540A6606740A42
:1001000067006800E703E800A8026607820A050C9A
:1001100088004306A802060C88004307740A67009B
:1001200004006607F00A940A6607F00A970A660751
:10013000F00A0400E702900A670004006607A30AB9
:10014000E7029D0AF00A0B0C2400040C2900080C9D
:100150002A00DC0C270004006606B10AE702AB0A9D
:10016000F00A6700B30A6607BA0A6607BA0AE70325
:10017000B20AF00A47032003EA02A90AA402E9022C
:10018000A70A7B0CAB004307F00AD50CAC00430771
:10019000F00A0B0C8D004307D40A160C8E0043079F
:1001A000D40A010C2F00EB0A210C8D004307DF0A53
:1001B0002C0C8E004307DF0A020C2F00EB0A370CD1
:1001C0008D004307EA0A420C8E004307EA0A030C3B
:1001D0002F00EB0AF00A6B006C006D006E00480AFD
:0401E0006F00EB0AB7
:021FFE00EE0FE4
:00000001FF
